:10000000992800000000000018288207FE34FD3403
:10001000FB34F734C03066001030650003306200F6
:10002000A0308B00F4309200063093009A01080053
:100030009500030E9600900A1008033991000C3EBB
:1000400084000008850011080520A00006080F386C
:1000500020058600920B34283A20F4309200930B4E
:10006000342806309300920A160E8300960E160E60
:100070000B110900141C08008C030C0F4C280930CC
:100080008C008D030D0F4C2805308D008E030E0F54
:100090004C2809308E008F038C08031D08008D0842
:1000A000031D08008E08031D08008F08031D0800AB
:1000B0009401191408008900831608148312080893
:1000C000080001301A075B208C0002301A075B2001
:1000D0008D0003301A075B208E0004301A075B2066
:1000E0008F00080083168801081555308900AA3052
:1000F0008900881488187A280815081283120800C5
:100100000C08880001301A07890072200D08880049
:1001100002301A07890072200E08880003301A077F
:10012000890072200F08880004301A0789007220A5
:1001300008000A20612014101910C020C620CC200D
:10014000861FA728061FD228051E1829A028C02010
:10015000F430920081011414861F9A281918B128CE
:10016000AC28061286163521061686123521861B06
:10017000B1282821861BB12806128612C0209A2891
:10018000861FC0282821861FC0280800061FC628F1
:100190002821061FC6280800051ECC282821051E78
:1001A000CC280800C6200A308F008E008D008C00FD
:1001B0008F01323097002821061FE628970BDB2895
:1001C0008F0A0A300F020319D828D928C6208E01B9
:1001D000323097002821061FF528970BEA288E0A4F
:1001E0000A300E020319E728E828C6208D013230B4
:1001F00097002821061F0429970BF9288D0A06303D
:100200000D020319F628F728C6208C01323097001A
:100210002821061F1329970B08298C0A0A300C0283
:100220000319052906298B1380208B17C620A028C7
:1002300004309A073C301A0203199A0100308900F1
:100240001A0888008B1372208B176120CC20A028FD
:1002500020309800F83031210000980B2A2908003E
:10026000F930FF3E031D312908003F30FF3E031DDA
:040270003629080023
:1042000000000100000000000000020000000000AB
:104210000000030000000000000004000000000097
:104220000000050000000000000006000000000083
:10423000000007000000000000000800000000006F
:104240000000090000000000000000000100000064
:104250000000010001000000000002000100000059
:104260000000030001000000000004000100000045
:0A427000000005000100000000003E
:00000001FF
